:100000000C9446000C9463000C9463000C94630001
:100010000C9463000C9463000C9463000C946300D4
:100020000C9463000C9463000C9463000C946300C4
:100030000C9463000C9463000C9463000C946D06A4
:100040000C9463000C9463000C9463000C946300A4
:100050000C9463000C9463000C9463000C94630094
:100060000C9463000C9463000C9463000C94630084
:100070000C9463000C9463000C9463000C94630074
:100080000C9463000C9463000C94630011241FBE55
:10009000CFEFD0E1DEBFCDBF11E0A0E0B1E0EAE4F8
:1000A000F7E100E00BBF02C007900D92AE32B1073E
:1000B000D9F711E0AEE2B1E001C01D92AA33B10759
:1000C000E1F70C9497060C9400002F923F924F9208
:1000D0005F926F927F928F929F92AF92BF92CF92D8
:1000E000DF92EF92FF920F931F93CF93DF93CDB7E1
:1000F000DEB726970FB6F894DEBF0FBECDBF5C010A
:100100006A017B01522E180127FF02C0552405C049
:1001100085E2821714F485E2582ED5019896BE83A5
:10012000AD8320E030E040E050E0C701B6010E941E
:10013000DE09882354F4F1018081918182609183EA
:100140008083F7FAF094F7F8F094AE014F5F5F4FB9
:10015000C701B6010E943E0A3B014C01E980FA80CA
:100160000B811C8120E030E040E050E0C801B70185
:100170000E94DE098823E9F1CD80DE80442428C076
:100180002DEC3CEC4CEC5DE3C801B7010E946E0A1B
:10019000AE014F5F5F4F0E943E0A2AE939E941E212
:1001A00051E40E946E0A0E94C309605DD6016E93FD
:1001B0006D014394E980FA800B811C8120E030E0DE
:1001C00040E050E0C801B7010E94DE09882319F021
:1001D000AC14BD04A8F2750106C0F60181916F014F
:1001E000D7018D937D01ED81FE81CE16DF06A8F348
:1001F00029C020E030E040E050E0C401B3010E949B
:10020000E10918161CF0750144241CC0442403C0E5
:100210004A943701480120E030E040E251E4C40153
:10022000B3010E946E0A7B018C0120E030E040E8BF
:100230005FE30E94DE0987FDEBCFE982FA820B8340
:100240001C837501D1014D915C9153FF13C0BDEF2B
:100250004B1684F0242D332727FD3095852D9927C3
:1002600087FD909501962817390724F45460F10111
:1002700051834083D1018D919C9192FD08C053948C
:10028000052D112707FD10950A0D1B1D0CC0052D0E
:10029000112707FD10950A0D1B1D842D992787FD39
:1002A0009095080F191F0A151B05D8F4F5014CC0CD
:1002B00020E030E040E251E4C401B3010E946E0A44
:1002C000AE014F5F5F4F0E943E0A3B014C016981C6
:1002D0007A818B819C810E94C309605DD7016D93F7
:1002E0007D010E151F0528F0ED81FE81EE16FF063B
:1002F000F8F28D819E810817190718F0F50117A2F1
:1003000024C0D8018C918B5F8C93F80131E318C025
:1003100020E3D8012C93A016B10628F48E918D010C
:100320008F5F8C930DC0D8013C934394D1018D9184
:100330009C9192FF05C0AE16BF0608F4208331964B
:10034000D8018C918A3324F71082842D992787FD58
:10035000909526960FB6F894DEBF0FBECDBFDF9105
:10036000CF911F910F91FF90EF90DF90CF90BF90B2
:10037000AF909F908F907F906F905F904F903F9045
:100380002F9008952F923F924F925F926F927F929B
:100390008F929F92AF92BF92CF92DF92EF92FF9295
:1003A0000F931F93CF93DF93CDB7DEB7EE970FB6C2
:1003B000F894DEBF0FBECDBFCC24DD2476013C0116
:1003C0007EAF6DAF5A011A821982FC011782168224
:1003D000838181FDF3C38FEF9FEF16C409811A81DA
:1003E00000FFD3C3842D80538A30D0F4F0E34F163E
:1003F00031F4552021F403FD02C0116075C18AE07B
:10040000252D2802C0011124542C580E30ED530E16
:1004100057FE02C04FE7542E03FDCAC3352CC8C394
:10042000442D45564CAF433028F0842D85548330FD
:1004300008F0FCC0C501049698AF8FABF501C080F1
:10044000D180E280F38003FD02C036E0532E077BAB
:100450001A83098346015701A7019601C701B60116
:100460000E94E9068823C1F08EE48D838B8381E4AA
:100470008C839E012A5F3F4F3AAF29AF3CAD3330AA
:1004800008F07AC28B81805E8B838C81805E8C8346
:100490008D81805E8D8370C2C701B6010E94350ACE
:1004A000892BE9F089E48D838EE48C8386E48B8349
:1004B00020E030E040E050E0C701B6010E94DE09D4
:1004C00087FD06C0AE014A5F5F4F5AAF49AFD6CF36
:1004D0008DE28E83CE0107969AAF89AFCFCFC80148
:1004E00092609A838983E7E44E1609F449C0E415C3
:1004F00044F0F5E44F1679F026E4421609F042C3C1
:100500001DC036E64316D1F047E64416C9F155E65C
:10051000451609F037C38E010F5F1F4F252DB5011A
:10052000A401CE010F960E946500282E8CEF380E94
:1005300015140CF43A94DE011F9615C094609A834A
:1005400089838E010F5F1F4F252DB501A401CE01B8
:100550000F960E946500282E15140CF43A94DE01C3
:100560001F96121444F4FD0101900020E9F7319721
:10057000CE2ECA1A02C0C52CC394BAAFA9AF7DC192
:10058000552011F0252D01C021E098609A838983C0
:100590008E010F5F1F4FB501A401CE010F960E947F
:1005A0006500282E89819A8192FF1EC0822D850DBB
:1005B0008150282FA82FBB27A7FDB095AC0FBD1FDA
:1005C0001F9605C08C9111972150803331F4622F12
:1005D00027FD23C02215B4F703C3C62E562E52188A
:1005E000539400C3C92E17C0252DE52DFF27E7FD25
:1005F000F095EC0FFD1F3F9606C080813197292FA3
:100600002150803379F7922F1216BCF3522EC22E4E
:10061000222309F4EFC2592EEDC2E22FFF27E7FD96
:10062000F095EC0FFD1F108A552499CFC8018870F2
:10063000907003FF04C0552011F421E0522EE9E62A
:100640004E1609F493C0E4153CF1F3E54F1609F496
:1006500074C0F415ACF02BE24216E1F1241544F01D
:1006600030E24316D1F143E2441609F080C23FC0A4
:100670005DE24516C1F18EE2481609F078C239C034
:1006800093E64916E1F1E4E64E1609F46FC0F8E589
:100690004F1609F06CC29FC020E7421609F496C0BD
:1006A000241544F03CE6431641F14FE6441609F0A8
:1006B0005EC20DC055E7451609F48FC0E8E74E1637
:1006C00009F489C0F3E74F1609F051C221C028E0B0
:1006D0002BAF83C000611A83098389819A8180626C
:1006E0009A83898365C200681A83098361C20064A2
:1006F000FBCF08601A83098352C20460F5CFA501BD
:100700004E5F5F4F58AF4FABF501C0803A9434C194
:10071000F501C080D180892B41F0652D772767FDD9
:100720007095C6010E94CC0718C0F6010190002008
:10073000E9F73197EC19EBAF11C0F501C080D1801A
:10074000892B41F0652D772767FD7095C6010E94C2
:10075000C10703C0C6010E94B8078BAF95012E5F89
:100760003F4F38AF2FAB3BAD331A06C102FF0BC072
:10077000A5014C5F5F4F58AF4FABF50160817181B0
:10078000828193810EC095012E5F3F4F38AF2FAB12
:10079000F501808191819C01B901882777FD8095C1
:1007A000982F6B017C0197FF0BC002601A830983AD
:1007B000F094E094D094C094C11CD11CE11CF11CB5
:1007C00089819A818F7B9A83898327C000641A83E9
:1007D000098398E7492E30E13BAF29813A8122FF16
:1007E0000BC0A5014C5F5F4F58AF4FABF501608167
:1007F0007181828193810CC0A5014E5F5F4F58AF1C
:100800004FABF50180819181AC01BA01882799270E
:100810006B017C012F7C3A83298387017601CE010D
:1008200003969AAF89AF9BADA92EBB24CC24DD24BF
:10083000C801B701A60195010E944C0B6A301CF05B
:10084000640D615201C0605DE9ADFAAD6193FAAF2C
:10085000E9AFC801B701A60195010E944C0B7901CF
:100860008A01211531054105510511F7CC24DD24FC
:100870007601CE010396C9ACC81A49815A81CA01D2
:1008800082739070892B09F03A9446FF07C0FBAD44
:10089000F03111F482E001C081E0381A43FF10C04A
:1008A000252D332727FD30958C2D99278217930707
:1008B00024F0477F5A83498303C05C18351801C070
:1008C0003C1840785170452B69F4832D06C0B30164
:1008D00080E290E00E942708812F182F11501816EF
:1008E000B4F3312E89819A8181FF04C0B3018DE276
:1008F00090E00BC084FF04C0B3018BE290E005C020
:1009000085FF05C0B30180E290E00E94270889813D
:100910009A8186FF0FC0B30180E390E00E94270810
:100920002BAD203139F4B301842D992787FD9095A3
:100930000E94270889819A8190FF0DC0832D06C0EF
:10094000B30180E390E00E942708812F182F1150F7
:100950001816B4F3312E89819A8183FF0DC0252D9D
:1009600006C0B30180E390E00E942708212F122FD8
:1009700011501216B4F3512E898187FD0DC0832DBD
:1009800006C0B30180E290E00E942708812F182F53
:1009900011501816B4F3312E33E6431631F4B30177
:1009A0008C2D992787FD9095BEC043E74416B1F47E
:1009B000460156011BAD09C0F50181915F01B301EC
:1009C000992787FD90950E9427081150A8F7640188
:1009D000FBADCF0ED11C2FEF2BAFB8C033E54316C4
:1009E000B1F446018601BBAC08C0F8018491B301A3
:1009F00099270E9427080F5F1F4FBA94FFEFBF1679
:100A0000A1F764012BADC20ED11CFBAF9FC0898141
:100A10009A8191FD03C009AD1AAD91C092FF1DC02E
:100A20001214BCF4A9ACBAAC122D09C0F501819125
:100A30005F01B301992787FD90950E942708115007
:100A4000A8F729AD3AAD220D311D3AAF29AF2224C6
:100A50000FC0B30180E390E009C0E9ADFAAD819128
:100A6000FAAFE9AFB301992787FD90950E94270857
:100A700015142CF4B3018EE290E00E9427088981BE
:100A80009A8192FD06C017C0B30180E390E00E94F6
:100A900027082394822D815087FF0DC05A94852DFD
:100AA0008F5F18168CF307C0B301892F992787FD34
:100AB00090950E942708E9ADFAAD9191FAAFE9AFA0
:100AC000992329F05A94852D8F5F18166CF389812C
:100AD0009A8192FD3BC0B301842D992787FD9095A3
:100AE0000E9427082A9427FE07C0B3018DE290E0F8
:100AF0000E942708219405C0B3018BE290E00E9478
:100B000027086AE070E0822D992787FD90950E9462
:100B1000390B6B017C01CB01C096B3010E94270801
:100B2000B301C701C0960E94270810C0F801829146
:100B30008F01B301992787FD90950E942708CE0168
:100B400003960817190791F71AAF09AF898187FF34
:100B500017C0832D06C0B30180E290E00E942708F1
:100B6000812F182F11501816B4F3312E09C0B3017C
:100B7000842D992787FD90950E942708B8AEAFAACB
:100B80001A821982AFA8B8AC13C0F5E24F1649F427
:100B900081E090E09A8389832AE02BAF33245524A7
:100BA00007C0B301842D992787FD90950E942708DF
:100BB0004DAD5EAD4F5F5F4F5EAF4DAFF3018381D3
:100BC00083FF04C0EDADFEAD449003C0EDADFEADBE
:100BD0004080442009F002CCF3018681978114C043
:100BE000C22E5524EC2DFF27E7FDF095EC0FFD1FDD
:100BF000108AB2CCEC2DFF27E7FDF095EC0FFD1F1E
:100C0000108AFEEF4F0E92CCEE960FB6F894DEBF30
:100C10000FBECDBFDF91CF911F910F91FF90EF904D
:100C2000DF90CF90BF90AF909F908F907F906F900C
:100C30005F904F903F902F90089510926100109216
:100C4000620080E487B987EE86B9089597B1907EF7
:100C50008770982B97B90895349BFECF0895349AE6
:100C6000089584B195B108950F931F93CF93DF93A7
:100C7000062F0E9426060E942F060E942C060E9424
:100C80002F06002319F4C0E0D0E00EC0C0E0D0E091
:100C900010E00E942C060E943106C80FD91F0E9446
:100CA0002F061F5F0117A9F7602F7727CE010E943B
:100CB000250BCB01DF91CF911F910F9108959C01DE
:100CC00012BE10922F0110922E0180912E01909150
:100CD0002F0182179307C9F708951F920F920FB63D
:100CE0000F9211248F939F9380912E0190912F0149
:100CF000019690932F0180932E019F918F910F90D9
:100D00000FBE0F901F90189513BE86B7836086BFE5
:100D100087B7836087BF8DE083BF12BE8DE781BF39
:100D200008955D9BFECF8CB980E090E00895CFEFF1
:100D3000D0E1DEBFCDBF0E9484061092900087E60E
:100D400089B988E08AB9789460E070E081E996E03A
:100D50000E94D70780E091E00E9474080E941D065F
:100D60000FE011E084E690E00E945F0665E080E01D
:100D70000E943406EC01BE01882777FD8095982FEC
:100D80000E94FB0ADD2334F420E030E040E857E421
:100D90000E94B70A20E030E040EA50E40E946E0A68
:100DA00020E030E040E85AE30E946E0A9F938F9360
:100DB0007F936F93DF93CF931F930F930E945408F9
:100DC0008DB79EB708960FB6F8949EBF0FBE8DBF25
:100DD000C9CFA8E1B0E0EFEEF6E00C947E0B69839A
:100DE0007A838B839C832D833E834F835887BE01F8
:100DF000675F7F4FCE0101960E941907BE016F5EAB
:100E00007F4FCE0105960E9419078985823018F41C
:100E100081E090E00AC020E030E08989823010F063
:100E2000C90103C021E030E0C901E2E068960C94FA
:100E30009A0BFC01DB01208131819281492F4F7790
:100E400050E0991F9927991F8381682F660F692B9E
:100E5000881F8827881FFD018183662309F049C008
:100E6000211531054105510509F470C082E89FEF55
:100E7000FD0193838283220F331F441F551F220FCE
:100E8000331F441F551F220F331F441F551F220FAE
:100E9000331F441F551F220F331F441F551F220F9E
:100EA000331F441F551F220F331F441F551F83E05C
:100EB0008C932030F0E03F07F0E04F07F0E45F074D
:100EC00090F482E89FEF220F331F441F551F0197B4
:100ED000203060E0360760E0460760E4560798F38C
:100EE000FD0193838283FD012483358346835783E9
:100EF00008956F3F71F1862F99278F579040FD011C
:100F00009383828383E08C93220F331F441F551FEA
:100F1000220F331F441F551F220F331F441F551F1D
:100F2000220F331F441F551F220F331F441F551F0D
:100F3000220F331F441F551F220F331F441F551FFD
:100F400050642483358346835783089582E08C93CD
:100F50000895211531054105510519F484E08C935C
:100F6000089544FD02C01C92BECF81E08C93BBCF9C
:100F7000FC0105900020E9F7809590958E0F9F1F4A
:100F80000895FC010590615070400110D8F78095DC
:100F900090958E0F9F1F0895FC0161507040019045
:100FA0000110D8F7809590958E0F9F1F0895EF92AE
:100FB000FF920F931F93CF93DF938C017B01892BBB
:100FC00011F4672BD1F16EE070E081E090E00E94B7
:100FD000A708FC01009789F1DC0180E88383E11414
:100FE000F10471F0F386E28681E883838091300119
:100FF00090913101892B21F4F0933101E09330017C
:1010000001151105E1F011870087838182608383D8
:101010008091320190913301892B89F4F09333014F
:10102000E09332018091340190913501892B39F49C
:10103000F0933501E093340102C0A0E0B0E0CD01AF
:10104000DF91CF911F910F91FF90EF9008950F9333
:101050001F93CF93DF938C01EB018B81992781FF45
:101060001BC082FF0DC02E813F818C819D8128177E
:10107000390764F4E881F9810193F983E88306C0B4
:10108000E885F985802F0995892B31F48E819F8120
:1010900001969F838E8302C00FEF1FEFC801DF917F
:1010A000CF911F910F910895CF93DF93CDB7DEB706
:1010B00022970FB6F894DEBF0FBECDBFFE01379664
:1010C00061917191FA83E983AF018091320190912E
:1010D00033010E94C20122960FB6F894DEBF0FBE04
:1010E000CDBFDF91CF9108950F931F93CF93DF93DF
:1010F0008C01E0913201F0913301838181FF1FC0A7
:10110000C0E0D0E00AC0FD0120853185BD01F901B4
:101110000995892B11F0CFEFDFEFF80181918F0155
:10112000A0913201B0913301882369F7FD01208538
:101130003185BD018AE0F9010995892B11F0CFEFC6
:10114000DFEFCE01DF91CF911F910F9108950F93A3
:101150001F93CF93DF93869F8001879F100D969FEB
:10116000100D1124C8010E94C308EC01009729F05A
:10117000A80160E070E00E94BC09CE01DF91CF9130
:101180001F910F910895CF93DF93AC01029710F454
:1011900042E050E0A0913801B0913901FD01C0E07A
:1011A000D0E020E030E020C0808191818417950755
:1011B00069F482819381209719F09B838A8304C00C
:1011C0009093390180933801CF0132C048175907F5
:1011D00038F42115310519F08217930708F49C01A2
:1011E000EF010280F381E02D3097F1F621153105F2
:1011F00089F1C901841B950B049708F4A901E0E06B
:10120000F0E026C08D919C91119782179307E9F425
:101210004817590779F4ED018A819B81309719F0BD
:101220009383828304C09093390180933801CD0168
:10123000029649C0841B950BFD01E80FF91F4193ED
:10124000519302978D939C933AC0FD01A281B38183
:101250001097C1F68091360190913701892B41F4A6
:101260008091290190912A01909337018093360152
:1012700020912B0130912C012115310541F42DB71E
:101280003EB78091270190912801281B390BE091EE
:101290003601F09137012E1B3F0B2417350788F0DC
:1012A000CA0102962817390760F0CF01840F951FF5
:1012B0000296909337018093360141935193CF0169
:1012C00002C080E090E0DF91CF910895CF93DF934B
:1012D000009709F44EC0EC0122971B821A82A0915C
:1012E0003801B0913901109711F140E050E001C090
:1012F000DC01AC17BD0700F1BB83AA83FE0121917D
:101300003191E20FF31FEA17FB0771F42E5F3F4F95
:101310008D919C911197820F931F99838883FD0172
:10132000828193819B838A834115510559F4D0931F
:101330003901C09338011DC0FD0182819381AD0147
:101340000097B1F6FA01D383C28321913191E20F64
:10135000F31FEC17FD0769F42E5F3F4F88819981D9
:10136000820F931FFA01918380838A819B819383EB
:101370008283DF91CF910895DC0101C06D934150CC
:101380005040E0F7089597FB47D09F3738F0FEE9CB
:10139000F91B982F872F762F6B2F05C05AC0969573
:1013A000879577956795F150D0F73EF490958095A5
:1013B000709561957F4F8F4F9F4F08950ED05EF0CF
:1013C00004C00BD026F001C008D019F020F48FEF34
:1013D000089580E0089581E0089597FB092E052681
:1013E00000F8689410D0E89407FC07C062177307F0
:1013F0008407950721F008F40094079498940895C1
:10140000052E092607FA440F551F5F3F79F0AA27DA
:10141000A51708F051E04795880F991F9F3F31F0BD
:10142000BB27B91708F091E0879508959F919F9188
:10143000112408C197FB880F991F9F3F31F0BB27EC
:10144000B91708F091E0879508959F919F91112415
:10145000F9C0662777278827992708959F3F59F471
:10146000803C49F481E09927089590688923872377
:1014700086238395B9F3882799270895DBDFCF93D7
:10148000DF93D52FC42F55274427332722279923AD
:10149000D9F09F37C8F0F92FBDD0592F482F372FDB
:1014A000262FF63968F46FDFA6D0C030CD0721F0C3
:1014B00069937993899399939058DF91CF9157C00D
:1014C0009927882777276627C030CD0721F02993F1
:1014D000399349935993DF91CF919CC091DF01D00B
:1014E00099C0992339F0552329F09F575F57950FDD
:1014F00013F49AF1B1CF91589F3FE1F3629FA12D70
:101500000F92BB27639FA00DB11DEE27729FA00D08
:10151000B11DEE1FAF93AA27649FB00DE11D739F0D
:10152000B00DE11DAA1F6627829FB00DE11DA61F09
:101530005527749FE00DA11D551F839FE00DA11D30
:10154000561F849FA00D511D852F7A2F6E2F1F903F
:101550000F9088231AF4939539F474C0000C111C71
:10156000BB1F661F771F881F012808955058192E2A
:1015700047DF01D04FC0BA1762077307840795078A
:10158000B1F188F40EF410940B2EBA2FA02D062E74
:10159000622F202D072E732F302D082E842F402DE3
:1015A000092E952F502DFF275523B9F0591B49F0CF
:1015B000573E98F0469537952795A795F040539557
:1015C000C9F776F0BA0F621F731F841F30F4879536
:1015D00077956795B795F040939517FA0F2E089574
:1015E000BF1BBB27BA0B620B730B840BF6CFDEF667
:1015F00033CFE89403C097FB0EF4D8DEB62F672FE5
:10160000782F892F9EE9002405C09A95BB0F661F8D
:10161000771F881F11249923A1F08823B2F79F3FD9
:1016200059F0BB0F48F421F4002011F460FF04C00E
:101630006F5F7F4F8F4F9F4F881F9795879597F9C3
:10164000089507CF9FEF80EC0895AA1BBB1B51E1C3
:1016500007C0AA1FBB1FA617B70710F0A61BB70B22
:10166000881F991F5A95A9F780959095BC01CD01C7
:10167000089597FB092E07260AD077FD04D0E5DFF1
:1016800006D000201AF4709561957F4F0895F6F703
:10169000909581959F4F0895A1E21A2EAA1BBB1B1E
:1016A000FD010DC0AA1FBB1FEE1FFF1FA217B3072E
:1016B000E407F50720F0A21BB30BE40BF50B661F44
:1016C000771F881F991F1A9469F760957095809508
:1016D00090959B01AC01BD01CF0108952F923F92DF
:1016E0004F925F926F927F928F929F92AF92BF9232
:1016F000CF92DF92EF92FF920F931F93CF93DF93DE
:10170000CDB7DEB7CA1BDB0B0FB6F894DEBF0FBE3A
:10171000CDBF09942A88398848885F846E847D8487
:101720008C849B84AA84B984C884DF80EE80FD8089
:101730000C811B81AA81B981CE0FD11D0FB6F894FF
:0A174000DEBF0FBECDBFED0108951E
:10174A000A0A47503244313220546573740A0069D8
:10175A0072203D20253375203D2025352E33662005
:0E176A00566F6C74730D0020003A01000000F1
:00000001FF
